:1000000094C1DEC110C2FCCFFBCFFACFF9CFF8CF3D
:10001000F7CFF6CFF5CFB8C1F3CFF2CFF1CFF0CF16
:10002000EFCFEECFEDCF1027E80364000A00010008
:10003000001000011000010000000000000000009E
:100040000000202053657420746F20736176652052
:100050000A20202020696E20536C6F74002020201D
:100060002020202320202300202053657420746F3B
:1000700020636C656172200A2020202020536C6F61
:10008000740057616974696E6720466F722043611E
:100090007264004F4B00536176656420696E207373
:1000A0006C6F74203100536176656420696E207333
:1000B0006C6F74203200536176656420696E207322
:1000C0006C6F74203300536176656420696E207311
:1000D0006C6F74203400536176656420696E207300
:1000E0006C6F74203500536176656420696E2073EF
:1000F0006C6F74203600536176656420696E2073DE
:100100006C6F74203700536176656420696E2073CC
:100110006C6F74203800536176656420696E2073BB
:100120006C6F74203900536176656420696E2073AA
:100130006C6F7420313000636C656172656420738C
:100140006C6F74203100636C656172656420736C40
:100150006F74203200636C656172656420736C6F2C
:1001600074203300636C656172656420736C6F7416
:10017000203400636C656172656420736C6F742059
:100180003500636C656172656420736C6F74203632
:1001900000636C656172656420736C6F7420370056
:1001A000636C656172656420736C6F7420380063E2
:1001B0006C656172656420736C6F74203900636CC8
:1001C000656172656420736C6F7420323000415336
:1001D0004D5A2047726F75700041534D5A20477237
:1001E0006F75702E0041534D5A2047726F75702EF7
:1001F0002E0041534D5A2047726F75702E2E2E00DF
:100200005061737320596F757220436172640A3EA6
:10021000005061737320596F757220436172640AD4
:100220003E3E005061737320596F757220436172B6
:10023000640A3E3E3E005061737320596F75722010
:1002400043617264003E3E3E3E005061737320592C
:100250006F757220436172640A20202020202020C4
:1002600020202020202020203C003C3C3C3C005012
:1002700061737320596F757220436172640A3C3C4C
:100280003C005061737320596F7572204361726432
:100290000A3C3C005061737320596F7572204361B2
:1002A00072640A3C0063617264310063617264329B
:1002B000006361726433006361726434006361726D
:1002C0006435006361726436006361726437006391
:1002D0006172643800636172643900636172643111
:1002E00030002020446F206E6F74204D617463686D
:1002F00000204275742054686520436172640A20AE
:1003000020206964206973203E3E000001002D4ECC
:10031000414E000080C00A00040038000100820144
:100320000C030200860114030000F894EE27ECBBD6
:10033000F1E0FBBFEBBFE5BFF8E1F1BDE1BD8DE052
:10034000A2E0BB27ED938A95E9F780E094E0A0E670
:10035000ED930197E9F7E6E1F3E085919591009738
:1003600061F0A591B59105901590BF01F001059040
:100370000D920197E1F7FB01F0CFEFE5EDBFE4E06F
:10038000EEBFC0E6D1E0E3C1AA93BA93EA93EFB718
:10039000EA93AB2DC0D4A05ABE4FECB1EC93EDE084
:1003A000EB1521F4E1E0AE2EBB2404C0EDE0EB152B
:1003B00009F0B394E991EFBFE991B991A99118952A
:1003C000ACD47394BCD4BED4C0D4EBE07E1620F47D
:1003D00017D4E2E4F0E011C0EBE07E16F8F0A72DB0
:1003E0009AD4EAE0F0E008D5EA1B9E2EE92DB1D4BC
:1003F000A9D4ABD405D4E8E6F0E0FA93EA933AD472
:10040000AAD4FED3EDE5F0E0AAD4E7E0EA93E0E079
:10041000A8D4EEE6F1E096D420D49DD4E4E1E7152B
:1004200008F4772486C179D4EBD3E2E8F0E097D4DE
:10043000552499D448F49AD4FF93EF9365D3AF91A0
:10044000BF91EC935394F5CFDBD3E3E9F0E087D48D
:1004500092D475D4E130A0E0FA0779F4552483D41E
:1004600058F48DD4A050B04081D48BD4E6E9F0E0AC
:1004700076D481D45394F3CF5CC1E230A0E0FA0784
:1004800079F4552470D458F47AD4A25FBF4F6ED457
:1004900078D4E6EAF0E063D46ED45394F3CF49C144
:1004A000E330A0E0FA0779F455245DD458F467D41A
:1004B000A45EBF4F5BD465D4E6EBF0E050D45BD4D0
:1004C0005394F3CF36C1E430A0E0FA0779F4552411
:1004D0004AD458F454D4A65DBF4F48D452D4E6EC65
:1004E000F0E03DD448D45394F3CF23C1E530A0E0ED
:1004F000FA0779F4552437D458F441D4A85CBF4F97
:1005000035D43FD4E6EDF0E02AD435D45394F3CF7C
:1005100010C1E630A0E0FA0779F4552424D458F449
:100520002ED4AA5BBF4F22D42CD4E6EEF0E017D431
:1005300022D45394F3CFFDC0E730A0E0FA0779F45A
:10054000552411D458F41BD4AC5ABF4F0FD419D42E
:10055000E6EFF0E004D40FD45394F3CFEAC0E830D0
:10056000A0E0FA0771F45524FED350F408D40CD45B
:10057000FDD307D4E6E0F1E0F2D3FDD35394F4CFFA
:10058000D8C0E930A0E0FA0779F45524ECD358F448
:10059000F6D3A059BF4FEAD3F4D3E6E1F1E0DFD3BD
:1005A000EAD35394F3CFC5C0EA30A0E0FA0779F458
:1005B0005524D9D358F4E3D3A258BF4FD7D3E1D3AE
:1005C000E6E2F1E0CCD3D7D35394F3CFB2C0EB3013
:1005D000A0E0FA0771F45524C6D350F4D0D3A0504C
:1005E000B040D5D3E7E3F1E0BAD3C5D35394F4CF09
:1005F000A0C0EC30A0E0FA0771F45524B4D350F455
:10060000BED3A25FBF4FC3D3E6E4F1E0A8D3B3D318
:100610005394F4CF8EC0ED30A0E0FA0771F4552466
:10062000A2D350F4ACD3A45EBF4FB1D3E5E5F1E063
:1006300096D3A1D35394F4CF7CC0EE30A0E0FA0758
:1006400071F4552490D350F49AD3A65DBF4F9FD335
:10065000E4E6F1E084D38FD35394F4CF6AC0EF3053
:10066000A0E0FA0771F455247ED350F488D3A85C37
:10067000BF4F8DD3E3E7F1E072D37DD35394F4CF32
:1006800058C0E031A0E0FA0771F455246CD350F45F
:1006900076D3AA5BBF4F7BD3E2E8F1E060D36BD3A4
:1006A0005394F4CF46C0E131A0E0FA0771F4552429
:1006B0005AD350F464D3AC5ABF4F69D3E1E9F1E0A7
:1006C0004ED359D35394F4CF34C0E231A0E0FA07AB
:1006D00069F4552448D348F452D356D358D3E0EAAA
:1006E000F1E03DD348D35394F5CF23C0E331A0E0EC
:1006F000FA0771F4552437D350F441D3A059BF4FB2
:1007000046D3EFEAF1E02BD336D35394F4CF11C0A4
:10071000E431A0E0FA0769F4552425D350F42FD32F
:10072000A258BF4F34D3EEEBF1E019D324D3539446
:10073000F4CFE991EFBFF991E991B991A99199911C
:10074000899179916991F990199009901895E0E053
:10075000E8BBE7BBE5BBEFEFE4BBE2BBE0E0E1BB3E
:10076000EBB7F7D2E06CEBBFE0E0E5BFE0ECEABF4F
:10077000E0E0E9BFEBB9E0E9EAB9E6E8E0BDE0E0D6
:10078000E0BDE3E3E9B9E0E1EA9394D2789438D2AA
:10079000EEECF1E0E4D2EFD233D2E9EDF1E0DFD2DA
:1007A000EAD22ED2E5EEF1E0DAD2E5D229D2E2EFBA
:1007B000F1E0D5D2E0D224D25524D5D228F4D6D235
:1007C000A0E0A0835394F9CFAA2009F040C0E0E054
:1007D000F2E0C5D2DFD2E1E1F2E0C1D2DBD2E3E266
:1007E000F2E0BDD2D7D2DD24E0E1DE1660F4E6E32C
:1007F000F2E0B5D2DA92E1E0B4D2E5E4F2E0AFD2D1
:10080000C9D2D394F1CFEAE4F2E0A9D2E2E3F0E076
:10081000C6D2E0E1DE2EE0E0ED1560F4E6E3F2E0C2
:100820009ED2DA92E1E09DD2EAE6F2E098D2B2D22C
:10083000DA94F1CFEFE6F2E092D2ACD2E2E8F2E065
:100840008ED2A8D2E4E9F2E08AD2A4D2BDCFAA2403
:10085000552489D248F48AD2A4D2A050B040A3D261
:1008600009F443945394F5CFA1D281F4C9D1E5EAB8
:10087000F2E075D29ED2A0D240F4AD9B02C0AD98FA
:1008800001C0AD9A9CD28394F6CF9CD2A0D26BD2F9
:1008900048F46CD286D2A25FBF4F85D209F443944C
:1008A0005394F5CF83D281F4ABD1EBEAF2E057D287
:1008B00080D282D240F4AD9B02C0AD9801C0AD9A07
:1008C0007ED28394F6CF7ED282D24DD248F44ED2DD
:1008D00068D2A45EBF4F67D209F443945394F5CF16
:1008E00065D281F48DD1E1EBF2E039D262D264D2EB
:1008F00040F4AD9B02C0AD9801C0AD9A60D2839424
:10090000F6CF60D264D22FD248F430D24AD2A65D5C
:10091000BF4F49D209F443945394F5CF47D281F4A1
:100920006FD1E7EBF2E01BD244D246D240F4AD9B4C
:1009300002C0AD9801C0AD9A42D28394F6CF42D2A4
:1009400046D211D248F412D22CD2A85CBF4F2BD27F
:1009500009F443945394F5CF29D281F451D1EDEBAE
:10096000F2E0FDD126D228D240F4AD9B02C0AD9872
:1009700001C0AD9A24D28394F6CF24D228D2F3D1E9
:1009800048F4F4D10ED2AA5BBF4F0DD209F44394C0
:100990005394F5CF0BD281F433D1E3ECF2E0DFD105
:1009A00008D20AD240F4AD9B02C0AD9801C0AD9A06
:1009B00006D28394F6CF06D20AD2D5D148F4D6D146
:1009C000F0D1AC5ABF4FEFD109F443945394F5CF13
:1009D000EDD181F415D1E9ECF2E0C1D1EAD1ECD14D
:1009E00040F4AD9B02C0AD9801C0AD9AE8D18394AC
:1009F000F6CFE8D1ECD1B7D140F4B8D1D2D1C4D13F
:100A0000D2D109F443945394F6CFD0D181F4F8D0E5
:100A1000EFECF2E0A4D1CDD1CFD140F4AD9B02C038
:100A2000AD9801C0AD9ACBD18394F6CFCBD1CFD1C5
:100A30009AD148F49BD1B5D1A059BF4FB4D109F494
:100A400043945394F5CFB2D181F4DAD0E5EDF2E0DE
:100A500086D1AFD1B1D140F4AD9B02C0AD9801C0F9
:100A6000AD9AADD18394F6CFADD1B1D17CD140F464
:100A70007DD197D189D197D109F443945394F6CF7E
:100A800095D181F4BDD0EBEDF2E069D192D194D152
:100A900040F4AD9B02C0AD9801C0AD9A90D1839453
:100AA000F6CF90D14424662061F5AAD0E2EEF2E0C0
:100AB00056D18824EAE08E1650F4AC9B02C0AC9864
:100AC00001C0AC9AE4E6F0E06AD18394F3CF98D009
:100AD000E1EFF2E044D188246FD150F4AC9B02C026
:100AE000AC9801C0AC9AE4E6F0E059D18394F4CF1D
:100AF00087D0E0E6F1E026D1B0D0E8EEF3E04FD1C8
:100B0000AC98662444CEFFCF5F9BFECFECB1089536
:100B1000A991B991E991F99130962AF4E095F0956F
:100B200031966DE26D93E89480E197E20DD088EE06
:100B300093E00AD084E6992707D08AE005D06E2F8B
:100B400010D066276C9308956627E817F90720F000
:100B50006395E81BF90BC9F7662311F416F00895A5
:100B60006894605D6D930895FFE0FA95F1F708953C
:100B7000A7B3AF70A7BBC19AC098F6DFC29AF4DFE3
:100B8000A6B3C298F1DFC29AEFDFC298A7FDF5CFF6
:100B90000895A07FAB2BA8BBC29AE6DFC298E4DF22
:100BA0000895C198A7B3A76FA7BBB8B3BF70A881BA
:100BB000F0DFA881A295EDDFC19AABC0C29AD4DF65
:100BC000E6B3C298D1DFE07F0895CEDFF7DFAE2F26
:100BD000F5DFC198E295EA2B0895CADFE881B9D024
:100BE000EA57FE4FE081B5D0DF01E981B2D0EA0FCC
:100BF000FB1FF0D0C980E881E0938A012296089516
:100C0000B7DFE2E0E7D0B4DFECE0E4D0B1DFE1E071
:100C1000E1D0E0E0E0938A01CE2E0895EF93FF93B8
:100C2000A8816894AA3031F0E894C394E0918B01D4
:100C3000EC1558F4E0918A01EF5FE0938A01E0E05F
:100C4000EA93E0918A018DD02EF092DFC09AA881BC
:100C5000AA93A7DFFF91EF915CC01A93A981BA8193
:100C6000ED91A983BA831E2FE03019F01A93D6DFD5
:100C7000F5CF0EC01A93E981FA813196E983FA83A0
:100C80003197E4911E2FE03019F01A93C7DFF3CFAC
:100C9000188123960895AA27BB271197F1F7089585
:100CA000C198A7B3A76FA7BBB8B3BF70A88171DF06
:100CB000C19A2FC0C298C098E881E0938B0149D0B7
:100CC000E058FF4FE0938801E88143D0E054FF4FA4
:100CD000E093890181D080D07FD0DDDFE0E2EA932C
:100CE000DFDFD9DFE8E276D0D6DFE4E073D0D3DF10
:100CF000E5E870D0D0DFA7B3AF70A7BBC19A65DFBE
:100D0000E53011F0E0E005C033DFE6E063D078DFE6
:100D1000E1E021960895B0E008950A921A92FA92BD
:100D20006A937A938A939A93AA93BA93EA93FA93DB
:100D3000EFB7EA93E8ECF0E0FA93EA9351C0E72DBD
:100D4000F0E00895FA93EA930895EEE6F1E0FADF11
:100D5000DFCEF0E00895E4EFF1E0F4DF41C0F2DF30
:100D600089CFEA933ACFEEE05E160895E52DF1DFE4
:100D7000E05AFE4F0895E8ECF0E0E4DF31C0A52D25
:100D8000CACFE0814CD03CCFAE59BF4F0895E0E0D0
:100D900046D036CFE2E3F0E0D5DF22D031CFD2DF4C
:100DA0001FC00080ECCF2FD0E0150895EEE0E415D1
:100DB0000895AA9A88240895E5E08E160895E0E93A
:100DC000F1E0EDCFAA98AD98E1E06E2E08954424AD
:100DD00055240895EA93E5CE5EDFE0E3EA9360CF21
:100DE000E991F991309639F080ED97E00197F1F7AC
:100DF000A8953197C9F708951B2EBF2FF12D1A2EF4
:100E0000AE2FE12D0895E199FECFFF93FFB7F8943F
:100E1000AEBBBFBBE09AEDB3FFBFFF910895E19B6E
:100E200002C0A895FCCF9FB7F894AEBBBFBBE09AB9
:100E30008DB3E81719F0EDBBE29AE19A9FBF0895D0
:00000001FF
